:030000000219FDE5
:03000B000200AA46
:03002B000201656A
:03005B000202F8A6
:030073000202DEA8
:1000800002030406080C10182030406080040608A3
:100090000C10182030406080A0C000070F1F3F0DDB
:1000A0000D04050D050305030302C2AFC0D0C0E077
:1000B000206217E5256002E473E525F4F58A758B67
:1000C00000D262D0E0D0D0D2AF3285268AC262E5BB
:1000D00026F46035306803207210758B00D0E0D0B4
:1000E000D0C293C295C297D2AF32C293C295C29783
:1000F000206E0C206609740AD5E0FDE57E429075FD
:100100008B00D0E0D0D0D2AF32758A00C28DD262DF
:1001100001FF01B9306805206602D29301B9306849
:1001200005206602D29501B9306805206602D29793
:1001300001B9C29230680A2066077408D5E0FDD282
:100140009301B9C29430680A2066077408D5E0FDAF
:10015000D29501B9C29630680A2066077408D5E0C6
:10016000FDD29701B9C2AFC2AD53E6EFC0D0C0E037
:10017000D2D3D2AFC2CEE52A6007207449152A2116
:10018000C67800790020742EE580307E01F430E3DB
:100190000278FF53DACF207E0343DA20307E034318
:1001A000DA10C2D8C271E580307E01F430E3027902
:1001B000FFC3E89970CB306103752A18207403756A
:1001C0002A18885FD27020740DE52B6004152B214E
:1001D000D643DA01C2D82070024134A85F20610200
:1001E000C2702074367982B70431C3E894F04003BA
:1001F00074F0F8E8C4540F28F87984B70302411B5F
:10020000C313C3138721200802C313200A06C3C8DF
:1002100098F8411B28F8500374FFF88822E52D5404
:10022000066011E533C313C31324062522F52250BB
:10023000037522FF7882B60459852224A824C3E5D9
:100240002495644002A864C3E895664002A86688C5
:1002500025E56970024185C3E8AA699A5003E8FA66
:10026000E4F9EAC333FBE56BF45B29400D256AF83A
:10027000E56A6002156A400B41850AC3E56A9A5037
:1002800002056A78FF8826C26EC3E52694F840020C
:10029000D26EC3E52594404002D26420CF0AD0E05C
:1002A000D0D043E610D2AD32C2CF053A7801E52A6C
:1002B0006005307402152AC3E55F9401400575623C
:1002C0000041D4756300756C00E5622401F562504D
:1002D000037562FFD0E0D0D043E610D2AD32C2AF9A
:1002E000C0D053E67FC260759100855694855795BE
:1002F000759104D0D0D2AF32C2AF53E6EFC2ADC0D9
:10030000D0C0E0C0F0D2D3D2AFA8FBA9FCC2D83095
:100310007102615F53DACF207E0343DA10307E032F
:1003200043DA20D271E580307E01F420E3026136A9
:1003300088278928A18653DACF207E0343DA20302C
:100340007E0343DA10C2D8C271307402A172780001
:10035000E580307E01F430E302A172885FA15A5338
:10036000DACF207E0343DA20307E0343DA10C271F5
:10037000206102813853DACF207E0343DA10307EC9
:100380000343DA20C2D8D271885A895BC3E89558F2
:10039000F8E99559F97B007E087A00C3E8948CE966
:1003A00094005005755E00812A882178A2E6A82174
:1003B0006055C3E894C8E994005008E4D2E4FB7A9D
:1003C0000A8105C3E89468E994015008E4D2E3FB8C
:1003D0007A0F8105C3E894D0E994025008E4D2E290
:1003E000FB7A1E8105C3E894A0E994055008E4D285
:1003F000E1FB7A3C8105C3E89498E994085008E44D
:10040000D2E0FB7A787E00C3E8955CFCE9955DFD5F
:1004100030E70AECF42401FCEDF43400FD755E00D5
:10042000C3EC9AED9E5003755E01885C895D855A28
:1004300058855B597802A15AC3E89527F8E99528B1
:10044000F9307C02A13E307B02A13E307A02A13716
:10045000207502815BE9FDE8FC817AE9C313F9E8C4
:1004600013F8307902A137E9C313F9E813F83078AB
:0F04700002A137E9C313FDE813FC206126C3EC9A
:10047F00941CED940240028191ED7018C3EC94C866
:10048F0050120529C3E529940A5002A172755F0025
:10049F00D270A172E529600215297888E6F97400F7
:1004AF00207F087896B90302789EE624FAFEE4349A
:1004BF0000FFC3EC9EFCED9FFD9208B90310A2084C
:1004CF005007207609D27681DD307602C276A208F7
:1004DF005016B9030DECF42401FCEDF43400FD02C9
:1004EF0004F778007900A13EB90315EC33FCED3326
:1004FF00FDC3EC940AFCED9400FD50047C007D00DC
:10050F00C3EC94FFED9400400678FF7900A13EEC18
:10051F008575F0A4C5F0A2F733F879004003020502
:10052F005A78FF790002055AE9C313F9E813F83036
:10053F007C0EE9600278FFC3E81338F8E43400F961
:10054F00C3E894FFE99400400278FF885FD27020DF
:10055F006102A172741FF4552F4BF52FC274EB700B
:10056F0002D274752A18307403752A0A306102A1F9
:10057F008620740353DAFE207403752B06D0F0D057
:10058F00E0D0D0D2AD43E6103279010205B679033F
:10059F000205B6790A0205B6791E0205B67964021C
:1005AF0005B679C80205B67817E4D5E0FDD8FAD9B3
:1005BF00F6227A147B780205DD7A107B8C0205DD3A
:1005CF007A0D7BB40205DD7A0B7BC80205DD79025B
:1005DF00B27DE4C294D5E0FDD295D5E0FDC295D5AC
:1005EF00E0FDD294D5E0FDD293E576D5E0FDC29340
:1005FF007496D5E0FDD9D9EAF8D5E0FDD8FBDBCE6E
:10060F00C29422C37C007D0075F00005F0EA33FA36
:10061F00EB33FB50F6EB13FBEA13FAC3E9FFE8FEEB
:10062F00E89AF8E99BF95004EFF9EEF8B3EC33FCD4
:10063F00ED33FDD5F0DFEDF9ECF822E889F08A20F3
:10064F00D2D4F8A9F07B0030F70B7BFFF42401F82C
:10065F00E9F43400F9E88520F0A4ADF0F8E985203D
:10066F00F0A4AFF0FEED2EF974003FFA7C04C3EA5C
:10067F0013FAE913F9E813F8DCF48BF030F70AE812
:10068F00F42401F8E9F43400F9E889F0C2D4F8A9A8
:10069F00F0227882B604030206FCC3E55F940140A2
:1006AF00030206C6852224E4F545F546F547F548CD
:1006BF00F549C26D0206FC7882E6FCD26DE522F5A3
:1006CF0023783879C7AA40AB41C3EB13FBEA13FA7F
:1006DF00EC146013C3EB13FBEA13FAEC141460076A
:1006EF00C3EB13FBEA13FAD1128845894622C3E5FF
:1006FF00459523F8E5469400F9500CC3E89480E93A
:10070F0094FF401602072DC3E8947FE9940050032D
:10071F0002072D787F790002072D788079FF884AAC
:10072F00894B22E54A2547F8E54B3548F9854B209B
:10073F00E4300701F43549FA30E709C3EA94F04091
:10074F001502076BC3EA940F500302076B78FF790A
:10075F00FF7A0F02076B780079007AF0C3E52495D2
:10076F0064500AC374019524500B020789E54B208E
:10077F00E70E020789E54B30E706884789488A4923
:10078F002278A4E6FAC3E54A33F8E54B33F9D14AA8
:10079F00E930E70BC3E89480E994FF4013E1C3C34A
:1007AF00E8947FE994005002E1C3787F7900E1C3B8
:1007BF00788079FFE820E715C3E52398F84009C34F
:1007CF00E8940140030207EA78010207EAE8F424FB
:1007DF00012523F840030207EA78FF884C2278A509
:1007EF00E6FAA848A949D14AE930E70CC3E89401D1
:1007FF00E994FF401602081EC3E894FFE9940050E5
:10080F000302081E78FF790002081E780179FFE9BC
:10081F0020E715C3E54C98F84009C3E8940140035D
:10082F000208457801020845E8F42401254CF840F8
:10083F000302084578FF88242278FFC26420693DAF
:10084F00206A12D264C3E541940A4009C3E5259496
:10085F00405002C26479A1E76023E541601F74FF35
:0F086F008541F0848539F0306A0375F005A4F8EF
:10087E00C5F0600278FFC3E895675002A8678866E6
:10088E0022C3E5409440E5419401E566500314010E
:10089E00A0046002F566220208A82275E89022786C
:1008AE0083E6FFE5E820ECF7A8BDA9BE0573C3E516
:1008BE007394084052757300E9FA79A0E76044EA30
:1008CE007007E574601B0208E3C3E895746010E5D9
:1008DE00745006600C140208EF0460F90208EFE58C
:1008EE0074F574C394A8401B7564C0C3940540137B
:1008FE00756480C39405400B756440C39405400332
:10090E0075640075BB0122E5642410500274FFF576
:10091E00647982B70402213CC3A864E5249850028E
:10092E00A824C3E895664002A86688258826E57344
:10093E00B4070375BB1E22743279A687F0A4C5F0E6
:10094E00A2F733F8C3E895644002A864882288248D
:10095E00882588268867227540007541F022C2AF2F
:10096E0075C820A8CCA9CDAA3A30CF010A75C824E3
:10097E00D2AFAB3BAC3C883B893CC3E89BF8E99CCF
:10098E00206908F9306702418121DEAD3D8A3DF9CB
:10099E00EA9DFA600478FF79FFAE3EAF3F8B3E8C46
:1009AE003FC3EC9FFCC3E99CF542A83BA93CC3E8BE
:1009BE009EF8E99FF9C3E54113FBE54013FAE82AD7
:1009CE00F540E93BF54150067540FF7541FF412862
:1009DE00AA40AB41AC40AD417E047F02C3EB940410
:1009EE0040021E1FC3EB940840021E1FC3ED13FDF1
:1009FE00EC13FCDEF7C3EA9CFAEB9DFBEF6009C338
:100A0E00E913F9E813F8DFF7EA28FAEB39FB8A4025
:100A1E008B4150067BFF8B408B41C3EB94025002FF
:100A2E00D2673069047F0341537892E6FFC3E537FE
:100A3E00948240110FC3E53794A040010FC3EF9489
:100A4E000640027F057E05E541C4540FF9E541C419
:100A5E0054F0F8E540C4540F28F8C3E89EFAE99420
:100A6E0000FB4009C3EA9402EB940050047A02E4BE
:100A7E00FB41CDAA40AB41EBC4FEEAC4540F4EFC81
:100A8E00C3EA9CFAEB9400FBC3E813C313F8EA28FD
:100A9E00FAEB3400FB8A408B41C3EB94024002C256
:100AAE00677805EBC4FE7B00EAC4540F4EFAC3EA26
:100ABE0098FA4005C3940250027A027892E6FF300B
:100ACE00600241CD855256855357D26043E680C3AE
:100ADE00E49AF8E49BF93067026167E8FAE9FBD320
:100AEE00E913FDE813FC88528953C3EF9403603871
:100AFE00EF20E00DE82CF8E93DF9ECFAEDFB020BE6
:100B0E0022E828F8E939F9C3E82402F8E93400F9B3
:100B1E007AFE7BFFC3EF9403400E8A548B55884EAA
:100B2E00894F8C508D51619B885489558A4E8B4FBD
:100B3E008C508D51306920C3E53394034019E54242
:100B4E00A2E713F8E555F4240138400B20E70875A9
:100B5E0054FFF42401F555619BE8FAD3E813FC88A1
:100B6E0052C3EF94036020EF20E007E82CF8ECFA74
:100B7E006187E8282402F87AFEC3EF940340088ABE
:100B8E0054884E8C50619B88548A4E8C50E56BC3B2
:100B9E00335002646BF56B30600261A5753402D27E
:100BAE006043E680E52D54066026A840A941C3E9BE
:100BBE0013F9E813F8C2AF53E67F759100C3E498BA
:100BCE00F594E499F595759104D26043E680D2AF21
:100BDE0022D265754400752000306B0375204002EB
:100BEE000BFED265754400752040306B03752000F6
:100BFE00D2AF7801206722E52D54066002C265C38C
:100C0E00E541940540137802940540087803940555
:100C1E0040027806306902780A206019E5446015B2
:100C2E0030690AC3E53394034003D53406D2AFD2FC
:100C3E006C81D871ADD2AF0000C2AF206726E541FE
:100C4E00C3FB940F40027B0FEB240530730123305E
:100C5E006A02742820620123F93069027982E58BD9
:0F0C6E00C39940B50544E59E7005E59B020C7FD8
:100C7D00E59A5440B5200281C230690A08C3E89450
:100C8D000A400108812720650261FEC26553E67F97
:100C9D007591003067107594007595FE759104D2AD
:100CAD006043E68061FEAE40AF41C3E49EF594E43F
:100CBD009FF59581A9C3E5339402500261FE30651D
:100CCD000261FED80281D68127C26C53E67F7591F1
:100CDD0000855494855595759104854E56854F57CD
:100CED00D26043E680D2AFE52D54066008206A023B
:100CFD000533020D12306C0D206B0A20650715812E
:100D0D0015810215A722780030640530650278013F
:100D1D00E53775F007A4F9E5F028F5F0E9A2F01331
:100D2D00A2F113A2F213F537C394785003753778F7
:100D3D00C3E53795384008D266C293C295C2973045
:100D4D006002A14C855056855157D26043E68022F2
:100D5D00207D14C2AF754302C294D292D2AF759F5B
:100D6D0033759E00020F3EC2AF754302C294D296F8
:100D7D00D2AF759F33759E00020F3E307243207DBA
:100D8D0020C2AF754303900143757E10C297C29682
:100D9D00306204D295A1A6D294D2AF759E23020FD4
:100DAD003EC2AF754303900143757E10C293C2924C
:100DBD00306204D295A1C6D294D2AF759E22020F95
:100DCD003E207D17C2AF75430390011EC29730625E
:100DDD0002D295D2AF759E23020F3EC2AF7543036B
:100DED0090011EC293306202D295D2AF759E22023F
:100DFD000F3E207D11C2AF754304C292D296D2AF81
:100E0D00759E22020F3EC2AF754304C296D292D296
:100E1D00AF759E23020F3E307249207D23C2AF7500
:100E2D004305900132757E04C295C294306204D29E
:100E3D0093C142D292D2AF759F33759E00020F3E81
:100E4D00C2AF754305900154757E40C295C2943072
:100E5D006204D297C165D296D2AF759F33759E004D
:100E6D00020F3E207D1AC2AF754305900114C29545
:100E7D00306202D293D2AF759F33759E00020F3E42
:100E8D00C2AF754305900128C2953062E8D297D262
:100E9D00AF759F33759E00020F3E207D11C2AF7559
:100EAD004306C296D294D2AF759E23020F3EC2AFB7
:100EBD00754306C292D294D2AF759E22020F3E3078
:100ECD007242207D20C2AF754301900154757E4062
:100EDD00C293C292306204D297C1EAD296D2AF7554
:100EED009E22020F3EC2AF754301900132757E0402
:100EFD00C297C296306204D293E10AD292D2AF75F4
:100F0D009E23E13E207D16C2AF754301900128C29C
:100F1D0093306202D297D2AF759E22E13EC2AF7579
:100F2D004301900114C297306202D293D2AF759EE5
:100F3D0023C26622900112757E00C293C295C2979C
:100F4D00C292C294C296C26222788076090876094E
:100F5D000876040876FF0876030876FF08760708FA
:100F6D007603087601087601788C76010876FF08FD
:100F7D0076FF0876FF0876FF0876FF087603087679
:100F8D00FF0876FF0876FF0876250876D0087628C4
:100F9D000876500876040876FF0876020876000871
:100FAD00767A0876FF0876010876010876000876CD
:100FBD0003227887E6FFC272BF0302D2727888E6F9
:100FCD00C394036008C27DE630E102D27DC27E7813
:100FDD0089E630E102D27EC3EF94026008758E017E
:100FED00D273020FF7758E00C273227880E61490CB
:100FFD0000809378A4F67881E6149000809378A50C
:10100D00F67886E61490008D9378A6F6789CE675B2
:10101D0038FF75390CB402067538A075390AB4035A
:10102D000675388275390578A3E61490009A93F504
:10103D0069120F4122227896E6FA7897E6FB7888B6
:10104D00E6B40305C3EB940EFB307F047A007BFFFF
:10105D00C3EB9AFCC3948250027C827575000575B2
:0F106D00EC8575F0A4C3E5F0947D40F222D27FAC
:10107C0011431205A77A007B007C1012059DE55FD9
:10108C002AFA74003BFBDCF37C04C3EB13FBEA137E
:10109C00FADCF7FEC27F114322E5EF20E603752050
:1010AC00000520903DFFE520146006901FFF1460A2
:1010BC00009304600375EF1253D9BF7581C043FFD1
:1010CC008012059875EF0243B203E5B3240420E7C0
:1010DC000DF521E5B120E0068521B343B101120FD6
:1010EC004175800875A40075F1FF75D4F7759002F1
:1010FC0075A5FC75F2FC75D50075A0FD75A602757D
:10110C00F30275D60075B0FF75A70175F4FF75E293
:10111C0041E4F8F6D8FD756B01120F561215E978FB
:10112C00988676753001C2AF1205B11205C1120551
:10113C00A71205C81205A71205CF1205A7C2AF78D2
:10114C00FA79FA308307D9FBD8F7021C00120FBFCB
:10115C00120FF81142114378988676120F41758858
:10116C005075891275C82475910475D84075A822DC
:10117C0075B80275E690759B80759D00759A8075A3
:10118C009C0075D10E75BC5875BB0175BA1F75E8FE
:10119C0080120598D2AF1208A553DACF207E0343F4
:1011AC00DA20307E0343DA1043DA01C2D8C271125E
:1011BC0005B1D2617B037A0CE55E70077A0CDB0318
:1011CC000211491205A7207003021149C270E55F94
:1011DC00C3940240E1E52F541F856160F561B56051
:1011EC00D5DAD5C26153DACF207E0343DA20307EC4
:1011FC000343DA10C2D8C27178A2E67008D274E543
:10120C002F54E0F52FC2757529001205AC30740906
:10121C00C3E529940A4002D27512059D78023074F8
:10122C00027800C3E55F9840F0C2AF1205C1120509
:10123C00C11205C1D2AF1205B1754D007888E6B464
:10124C000302612612059D788CE6C39401500302BB
:10125C001326E530C394015003021326207435C3C2
:10126C00E55F94FF5003021326C2AF1205D6D2AF2E
:10127C001205ACC3E55F940150EFC2AF1205C11269
:10128C0005A21205C1D2AF1205ACC3E55F94FF40B5
:10129C00E90217917F02D27F11431205ACC2AFC293
:1012AC007F1143AE5FC3E55F947FD2AF40761205EA
:1012BC0098C2AF1205D6D2AFDFDC117AC3EE94051B
:1012CC007897F61205B112162B1217147F0AD27FDB
:1012DC0011431205ACC2AFC27F1143AE5FC3E55FD1
:1012EC00947FD2AF50E6120598C2AF1205C1120519
:1012FC00A21205C1D2AFDFD6117AEE24057896F68C
:10130C001205B112162B1217431205AC1143C3E58B
:10131C005F94FF50024168021791C3E55F954D4001
:10132C0003855F4D1205AC78017988E7B403027828
:10133C0005C3E55F9840024148C2AF1205D61205BD
:10134C00D61205D6D2AF1205B1753000E4F531F5E1
:10135C00320531E531F470390532789AE678191492
:10136C006012783214600D787D14600878FA14607D
:10137C0003753200C3E53298401715327531B478D5
:10138C00998676C2AF1205D6D2AF789886761205BA
:10139C00AC1205A2E52A70053074022149780120AF
:1013AC0074027806C3E55F9840A77888E6C3940377
:1013BC0060031205ACE52A7003021149C2AF120F8B
:1013CC0041E4F522F523F524F525F526F56AD2AF8F
:1013DC007885E6C333F568E4F545F546F547F548F9
:1013EC00F549F573F52CF52DF53775730875BB1E9E
:1013FC001205981208A9E5E820ECFBA8BDA9BEE9E6
:10140C007001F888741208AD75730875BB1E788767
:10141C00E6FE7602120FBF7887EEF6C2AF7564FF58
:10142C00120945852264852265852266D2AF752214
:10143C000175240175250175260185636C756D0197
:10144C007888E6B40307C27D307602D27DD268D2AA
:10145C0069753300120EA7120ECC12096512096CB5
:0E146C0012096512096C120965021485C2AFDF
:10147A00120FBFD2AF75730075BB01120BF01206C3
:10148A00A1120D13120D5D12096C120BDF306D03E0
:10149A001206FD20670312084830670312088F12EC
:1014AA000D13120D8812096C120BF0306D0312071E
:1014BA0032120D13120DFF12096C120BDF306D037D
:1014CA00120790120D13120E2412096C120BF0302F
:1014DA006D031207ED120D13120EA712096C1208F2
:1014EA00A9120BDF120D13120ECC1208AD12096CE1
:1014FA00306935206B3285676485676585636C75ED
:10150A006D0179187A0CC3E53399400FC269D26A22
:10151A008A35856764856766021532C3E55F94017B
:10152A0040030214850215AF306A1B206B18E5359B
:10153A00147004C26A8178F535C3E55F94014003EB
:10154A000214850215AF753600C3E56278FA985021
:10155A0054307404E52A604D7888E6B40317207D78
:10156A0005207607A17F307602A17F206B07D26B18
:10157A0085676481C478F0306B058567647820C319
:10158A00E5419850028185306B1BC26BC27D307673
:10159A0002D27DD26A75351285676481850536E582
:1015AA005F6002A1B2753600C2AF120F417887E6BA
:1015BA00FE7602120FBF7887EEF6E4F522F523F5E0
:1015CA0024F525F526F568C268D2AF120598120FE0
:1015DA0041307409C3E536940540022149615890A7
:1015EA001A0D782012166DE520B4550CA312166D4B
:1015FA00E520B4AA0302160B120F5612162B021676
:10160A002A901A0378807B0A12166DA308DBF990D8
:10161A001A0F788C7B1812166DA308DBF9901A271B
:10162A0022C2AF1216AC121686901A00740E121647
:10163A0072A37404121672A37414121672901A0307
:10164A0078807B0A121671A308DBF9901A0F788C3E
:10165A007B18121671A308DBF91216BF12169D9099
:10166A001A2722E493F622E6438F01538FFD75EF82
:10167A000275B7A575B7F1F0538FFE22438F024367
:10168A008F0175EF0275B7A575B7F1901A0DF05372
:10169A008FFC22901A0D7455D172901A0E74AAD129
:1016AA0072227A3079D07820901A40D16DE520F7ED
:1016BA0009A3DAF7227A3079D0901A40E7D1720971
:1016CA00A3DAF922AB77A878BB01027980BB0202C0
:1016DA007981BB03027982BB04027984BB05027952
:1016EA0086BB06027992BB07027987BB080279A3F7
:1016FA00BB0902799CBB0A027988BB0B027989E88B
:10170A00F7227C051205B1DCFB22C2AF1205C11219
:10171A0005C81205CF1205D61205A21205C1120577
:10172A00C81205CF1205D61205A21205C11205C8A4
:10173A001205CF1205D6D2AF22C2AF1205D61205B4
:10174A00CF1205C81205C11205A21205D61205CF7D
:10175A001205C81205C11205A21205D61205CF122A
:10176A0005C81205C1D2AF22AE77AF78C2AF120553
:10177A00C11205C11205C11205A2DEF21205D61266
:10178A0005A2DFF8D2AF22F114F10CF10C75770142
:10179A00757801757900F1727C05AD5F1205B1C3E8
:1017AA00ED955F70F5C3E55F9401400AC3E55F9468
:1017BA00FF40320217CDD1CED12BF114C2AF75EF53
:1017CA0012F10CDCD50579C3E5799403500280C681
:1017DA00F10C0578E5771490009F93F808C3E57833
:1017EA0098500280AEF10CF10C0577C3E577940CA2
:1017FA005002809C120F5612162BC2AF75EF1212AE
:02180A00170CB9
:0319FD000210A530
:101A00000E0414090904FF03FF0703010155AA018D
:101A1000FFFFFFFFFF03FFFFFF25D0285004FF0259
:081A2000007AFF01010003FF41
:101A400023506C6174696E756D31353041232020EF
:101A500023424C48454C4923463331302320202033
:101A60002020202020202020202020202020202076
:101C0000C2AFC2D353D9BF7581C043B20343FF8073
:101C1000752438752503B1C975EF0275E24043F1AB
:101C20000853A4F775D400D2837DFA780379E67C53
:101C300010752200752300901DD67B0675249875BB
:101C400025013083028142208308D8FBD9F9DCF7D3
:101C500081B4308308D8FBD9F9DCF781B4B189E4C9
:101C600093A3C39A6004DDC381B4DBDBB17B600264
:101C7000812B7B08E493FAA3B15CDBF87A30B15C8A
:101C8000752200752300B17BEAFCEBFDC3ED94FEE9
:101C9000400EB17B8A278B28ED30E0048A828B834B
:101CA000B17B7AC270D8C3ED94FE601350CEBD00F4
:101CB00025EC60097520007521FF0200008100A855
:101CC00027A9280809D804D90281D3B17FEA89AAB3
:101CD000F281C50D81A0C3ED94035049EDA2E092BD
:101CE000007AC5C3E5829400E583941C50902000DF
:101CF00010438F02438F0175B7A575B7F1F030001F
:101D00001FA827A9280809438F01538FFDD804D99C
:101D100002A12089AAE275B7A575B7F1F0A3A10DBC
:101D2000538FFC817C7AC1BD030CE493A3FAB140CC
:101D3000DCF8B138817C817EAA22AB23B15CEBFA5E
:101D4000EA6222752608C3E52313F523E52213F57D
:101D50002250066323A0632201D526EAB1C9B1C986
:101D600075260AEAF4200102D283300102C283B14F
:101D7000C9C3134002C201D526EB22B17FEAFB2082
:101D80008302A17F308302A184752608AE24AF258B
:101D9000C3EF13FFEE13FEB1CDB1C9C3EA13308315
:101DA000024480FA30E703632201C3E52313F523DD
:101DB000E52213F52250066323A0632201D526D91C
:101DC000E52265236523F52222AE24AF250E0FDE22
:101DD000FEDFFCD20122424C48656C693437316326
:041DE000F3100601F5
:00000001FF
